:1074000080E189BD82E189BD09B400FEFDCF089508
:10741000CCD569F08091E9008F931092E900A1D456
:1074200083FF01C020D58F9187708093E900089574
:107430008EEF0090E10008220092E1000895F20131
:10744000F999FECFF2BDE1BD0895F9DFF89A80B554
:1074500008C0F5DF1FBA80BD0FB6F894FA9AF99A02
:107460000FBE31962F010895E0E0F0E085919491F0
:10747000019608958AE28BB98BEA34D01092890084
:107480008AEF8093880082E080936F0083E080938E
:107490008100E7E5F7E785913AD0E336E1F781E04F
:1074A0008093D7008AE482BF1092D8001092E20045
:1074B0001092DA001092E10080E808D019BC1EBAE0
:1074C0001092E00064D489E055D481E98093D8001B
:1074D0000895A3E6B1E090E81AD08D939A95E1F76C
:1074E000089586E008D010C083E005D08F2F0FD01C
:1074F0008E2F0DD080E05B9A5A9809C005D085E0A8
:10750000FADF05D080FDFDCF5A9A5B9808958EBDB5
:107510008DB587FFFDCF8EB508958FE08221E9F705
:10752000F3DFE3E6F6E090EB5C98892FF0DF80E193
:10753000EEDF5C9A8191EBDF83E68E278F77D1F7C0
:107540009395983B89F70895E3E6F1E094FC36C003
:1075500097FC4DC092FE089596849920D1F3F8943B
:10756000C089D78520E030E080E090E4AFEFBFEF46
:10757000119689199040E0F72D01BD4F8D0127FD2F
:1075800013C0E0E0F8E011928EE7819392E4E117F6
:1075900091939AE508F092E4E334C9F7819310825D
:1075A000BFDFFE012196A0DF94DFF90101D520584D
:1075B0003F4F040D151D9A9411F710C28301282D19
:1075C00060906C0170906B0143D019F48823C1F76F
:1075D0000895380188243CD0C9F580916A0182174A
:1075E00009F4830160906E0170906D01F4CF80E822
:1075F000982E60906E0170906D012AD059F4882306
:10760000B1F708959FEF96FC03C095FE089591E0B1
:1076100097FB890E662477248301222719D0B1F4C1
:107620008823A1F380916A0136F0881650F48217FE
:1076300030F0213003C0881520F4281710F483019E
:10764000282F60906E0170906D01E8CF3801822E76
:10765000F3014ADF3EDFC3E6D1E0E0E5F7E709905A
:107660008591081621F4E735D1F7088080104CCFBA
:10767000C9E031DFCA95E9F7D0E194FC55C097FC29
:1076800037C095FE1AC0C3E6D2E0E3E6F6E098E024
:1076900088E78E0F00840192E817E1F7884F099080
:1076A0000192E817E1F7C858DF4F9A9589F735DF5F
:1076B000C85FD340C33E49F749C0C3E6D6E0EBE517
:1076C000FAE098E08E2F885702900086E817E1F7DD
:1076D00038960A900292E817E1F73897C857D040D9
:1076E0009A9581F71ADFC850DC4FC33E41F72EC090
:1076F000A3EEB6E0E3E6F6E09AE0C6E00D90808106
:107700008025807F802582958193A336B90709F46F
:10771000B2E0E336F90709F4F2E0E336FC0771F76B
:10772000FCDEDA9529F712C0A3EEB9E0E3E6FAE051
:1077300092E00E90829180258F70802582958083C3
:10774000E336F907B1F7E9DEDA9571F7882708958E
:1077500041524455424F59D5F08D14A1C881CFD91B
:10776000F1AF000000FFFFCFCFFFFFFFFFCFCFFF44
:10777000FF0000FE067E7E06FE46565616FE0656A4
:10778000461EFE3F61E9E3FFE3EBE3FFE3EBE3FFCC
:04779000E16B3F006A
:10779400120110010200000841233600010000001C
:1077A400000109023E0002010080320904000001C8
:1077B4000202010005240010010424020405240629
:1077C4000001070582030800FF09040100020A0002
:1077D40000000705040210000107058302100001E0
:1078000011241FBE04B714BE88E18093600010925B
:1078100060008EEF9AE09EBF8DBF222433242101A9
:107820003101410180E88AC00F928F939F931F928C
:107830000FB60F9211244F936F938091DA0080FF5F
:1078400037C023C00F920FB68F939F93EF93FF9390
:1078500088278093850080938400E0E5F1E09281A1
:10786000907261F490818917980B908309F45D9A66
:1078700091818917980B918309F4289A239411F424
:107880008315381EFF91EF9154C08091D80080FF7E
:107890000FC08091DA008E7F8093DA008091D9004A
:1078A00080FF04C0ADDD81E08EBB02C019BC1EBAF2
:1078B0008091E10080FF0BC057D280FF08C057D2F3
:1078C0008091D800806202DE19BC85E08EBB809179
:1078D000E10084FF1AC048D284FF17C091DD809177
:1078E000D8008F7DF3DD8FEEA4DD3ED28F7E8160E8
:1078F00041D280915301882331F48091E30087FDC8
:1079000002C081E001C084E08EBB8091E10083FF72
:107910000CC02AD283FF09C087EF8BDD82E08EBBCB
:107920001092530185DD23D232D26F914F910F9087
:107930001F909F918F910FBE0F90189580936100BB
:1079400010926100B1E0B5BF82E085BF81E985B9E1
:1079500087EE84B91DB8769A10BA83EF81BB8CE2AA
:107960008BB98FE38AB980E58CBDBDBDA0E0E4E9A9
:10797000F7E705900D92A035E1F71D92BB30E9F7CE
:10798000000004C07F9B02C06FDD41F573DD789479
:107990005FDE71F0ABE9B7E0E3E6F7E790E1059071
:1079A0000D929A95E1F7A059BF4FE339B9F7B9DDC8
:1079B0004FD02EDD80915201807861F48FB1809597
:1079C000807F66991C9B8460982E1CDE8110BCDD34
:1079D00092FC02C0332062F747DD51F3F89489EB43
:1079E00081DD81E08093E00010926F0010928100B1
:1079F000109285001092840081E085BF15BE5D9ACB
:107A0000289A0C940000ABD107C05ED102C0CDD241
:107A100039F0A7D182FFFBCF85FFF7CF8091F1002E
:107A20000895082E83E09CD185FD07C091D102C046
:107A3000BCD269F096D180FFFBCF0092F10080911B
:107A40005201807221F45D9884E68093500108957C
:107A500086D182FF3BC180915201807221F4289827
:107A600084E680935101CFDF182F853431F422242E
:107A70008EE7382EE4DC8DE012C1843511F4C3DFCB
:107A8000FACF8C34C1F38035B1F3843721F484E428
:107A9000C8DF80E004C1813611F489E500C181347A
:107AA00029F4B1DF582EAFDF482EE5CF803711F42F
:107AB00083E5F5C0833539F4E0E5F7E78591B1DF7B
:107AC000E735E1F7EDC0863521F482E3AADF80E3F4
:107AD000E6C0863781F481E3669B8E5F1C9B8F5FD7
:107AE000A0DF81E47C9B885F7D9B8C5F7E9B8E5FAB
:107AF0007F9B8F5FD4C08837C1F485DF80935201AC
:107B0000289A84FD28985D9A83FD5D9887FD8824D6
:107B1000877009F487602E9A81FD2E98589A82FD0D
:107B200058982D9A80FD2D98A6CF8A3649F48FE972
:107B3000E2DCC3E0ECDC75DFCA95E1F7E5DCB0C060
:107B4000833731F487E86DDF85E96BDF8EE1A7C00D
:107B5000853639F4E0E8F3E73ED2E058F040E0F74C
:107B60008ACF823631F489E55CDF80E05ADF80E835
:107B700096C0823419F0873609F07DC0332443DF84
:107B8000D82F41DFC82F3FDF082F8354843008F0FF
:107B900085C0063411F4440C551CF20110926F009C
:107BA0001736B9F4033489F483E09FDCB0DC8EB57A
:107BB0001EBC37DF0DB42197D1F7A6DC08C0063410
:107BC00011F4859101C041DC2CDF2197C2F72F0110
:107BD0004AC00334A9F4E11104C083DC88ED85DCDC
:107BE0008DDC7FDC82E081DC0EDF0DB48EBDCA95BA
:107BF000D9F731968DDC82DCDA9569F72F0131C037
:107C00000634F1F49F01F437D8F4E5D119C0FBDE56
:107C1000063461F4C0FB46F0F43728F4182E81E0F6
:107C200087BFE89511243296082E0AC0043439F42F
:107C3000DF01B370AD59B94F8D93319601C009DCA6
:107C400021972AF7043431F42F01F370FE2B49F405
:107C500068DC07C0063429F42F01F901F43708F471
:107C6000B8D18DE0DEDE063411F45694479482E0FC
:107C700080936F0015C08237E1E049F08634E0E080
:107C800031F08E34E3E019F0813531F4E2E0F0E0D8
:107C900089E087BF849103C08B3111F08FE3C1DE8F
:107CA00083E0C3DB55D095FF03C009C07ED171F0DE
:107CB00058D080FFFBCF4CD002C077D139F051D0E3
:107CC00080FFFBCF84E0B1DB8BE743C00895E4E5A0
:107CD000F1E067E090915B0180915C01913231F0BD
:107CE000913AE1F58132D1F55ED181C0823271F4F1
:107CF0008191805B8191844089F580915D0180FD57
:107D00002DC0F89481E08093E0007ACD803231F587
:107D10004AD14BD1E9F08530D9F023D083FD18C08A
:107D200082FFF7CF04C07ADE8193615031F09091E9
:107D3000F3008091F200892BB1F7C6DF611549F796
:107D400004C033D129F0853019F00BD080FFF9CF72
:107D50008EE79091E80089238093E800089584E0FD
:107D600064DB8091E80008958091E2000895FCDFD3
:107D70008E7F80618093E200089582E061EC09D0FB
:107D800083E061E802D084E060E842E103C080E083
:107D900060E042E04ADB81E007D01092ED006093A2
:107DA000EC004093ED0008959091EB00892B8093B7
:107DB000EB00089560E0923029F0913029F4E0E082
:107DC00062E102C0E2E16EE3F1E0089580915B01BF
:107DD00088234CF402C0E9D0C1F3C3DF82FFFBCF9C
:107DE00073CFE3D091F3BDDF80FFFBCFB1CF4091E4
:107DF0006101509162014617510520F0462F61152F
:107E000009F4A6DF50E022C0D0D061F1853051F1F5
:107E1000A8DF83FD59CFA5DF82FD21C080FF16C0FA
:107E20003091F3002091F20006C081918093F1001F
:107E300041502F5F3F4F411519F028303105A8F30D
:107E400050E02830310509F451E082DF4115E1F6B8
:107E50005523D1F604C0A9D029F0853019F081DF6F
:107E600082FFF9CF31CFEBE5F1E0D8DD8193E33646
:107E7000E1F72DDF76DF83FF91C080915B01909168
:107E80005C01913009F170F09330F1F0953009F414
:107E900044C0963009F456C0983009F460C0993057
:107EA00059F767C0823841F780915F01BDDA2091B0
:107EB000EB001092E90077D022952695217020934F
:107EC000F1001092F10052C0882311F08230A1F627
:107ED0008F71823089F680915D018823D1F42091E1
:107EE0005F01277049F22093E9008091EB0080FF49
:107EF00010C0933011F480E20BC080E155DF81E0C7
:107F0000880F2A95E9F78093EA001092EA0088E04A
:107F10004BDF1092E90047D02AC0882391F41091DA
:107F20005D0110680FB7F8943ED050DF1ADF80FF74
:107F3000FDCF1093E300103883E009F482E08EBB9C
:107F40000FBF2CC08058823048F580915D01909120
:107F50005E0130DF603011F126D049DF1FC080386C
:107F6000E9F421D0809153018093F100F1DE2EDFFE
:107F700015C0882399F490915D01923078F4909324
:107F8000530111D023DF80915301882321F4809184
:107F9000E30091E087FD94E09EBBEFDEE2DE83FF2D
:107FA000089580E201DF87EFD4CE8EB38823089551
:107FB000A3E6B1E0F437B8F40ED090E40D901D9034
:107FC00081E087BFE89532969A95C1F71124E05871
:107FD000F04085E001C083E001D081E187BFE895F2
:087FE00007B600FCFDCF089577
:067FFA003230DBCFFBDC9E
:040000030000740085
:00000001FF
